:020000040000FA
:06000000653003303A28D0
:08000800A000030EA100831209
:1000100005191028831601178312B23081002B288E
:1000200083160113831203140B190310A80DA90DD5
:10003000AA0DAB0DAC0DAC16FF302C02031D2B2806
:10004000FA302B02031D2B2831152A08AF0029088E
:10005000AE002808AD008B100B11210E8300A00EFE
:04006000200E090065
:0C007400203084008001840A80300402E7
:10008000031C3C281230B000972183160C308505E4
:1000900087018312850187010730990000309A009B
:1000A000103083168E008312603083168F00831207
:1000B0000030831691009F008312C83083168100A0
:1000C000831231309000003083168C008312103080
:1000D0008B00272281018E018F010B118B100B10D9
:1000E0008C018B17812031198420B30B7F280310DA
:1000F00085190314B90DF030390203190C21282297
:10010000722864003210080031110130B7008514E4
:100110008B132030370783169B001C141A08831298
:10012000A4001030370783169B001C141A08831292
:10013000A300A6000230A6060030370783169B00F6
:100140001C141A088312A200A7000130A7068B17FF
:10015000321CB02822090339A200A309A409A50969
:1001600024082F02031D062923082E02031DD82868
:1001700022082D02031D062901303702031DC32862
:100180003D143E14AC2102303702031DCA28BD14B1
:100190003E14B42103303702031DD1283D153E140F
:1001A000BC2104303702031DD828BD153E14C421DC
:1001B00026082E02031DFD2827082D02031D0629EF
:1001C00001303702031DE7283D103E14CC210230D8
:1001D0003702031DEE28BD103E14D4210330370230
:1001E000031DF5283D113E14DC2104303702031DA8
:1001F000FC28BD113E14E42106295F08F039A03C1B
:10020000031906292E1A06290529EC21B70A0530FB
:1002100037020318080088280130B600B300B40084
:10022000B500B70085018701B11311228120B30BFE
:100230004729031085190314B90DF0303902031949
:100240006E29B41F8501B41F8701B41F8510B40B3C
:100250004729B50B47290230B50001303702031991
:10026000F521023037020319FA210330370203194E
:1002700003220430370203190C223708B608031989
:10028000B600031945298514B603FA30B400311DB0
:1002900016293111321C51292D090339AD00AE093F
:1002A000AF092F1C16298E018F010C1C16290C106A
:1002B0002E1E16298B1320303707BB002F08BA00DB
:1002C000822110303707BB002E08BA00822100308F
:1002D0003707BB002D08BA0082218B171522850134
:1002E0008701B70AB60105303702031C16292722F9
:1002F00008003E1C08003E101030BB003D08BA004C
:10030000822108008B133A0883161C159A00831269
:100310003B0883169B0055309D00AA309D009C141D
:1003200064009C1890291C1183128B1708008316F7
:1003300000309B001C141A088312DF008316203043
:100340009B001C141A088312C1000130C11BC1009C
:10035000C1080319C10008000712871640084107A9
:10036000D0000F08D100080005128715400841078A
:10037000D2000F08D3000800071185164008410776
:10038000D4000F08D5000800071087144008410763
:10039000D6000F08D700080087120716400841074B
:1003A000D0000F08D100080087110516400841074A
:1003B000D2000F08D3000800851207154008410736
:1003C000D4000F08D5000800871007144008410723
:1003D000D6000F08D70008000712051207110710F2
:1003E000871287118512871008003F09303987006E
:1003F000BF000800380910398500B8003F090839E6
:100400008700BF000800380920398500B8003F097F
:1004100004398700BF0008003F0903398700BF0087
:100420000800B801BF01BF160800B801BF010130C4
:100430003702031D1C2ABF1502303702031D212A73
:10044000B81603303702031D262ABF14080008001F
:100450005F080F390A3C0319552A50084002031D52
:10046000372A51080F02031C372A07128712520835
:100470004002031D412A53080F02031C412A0512A2
:10048000871154084002031D4B2A55080F02031C14
:100490004B2A0711851256084002031D552A57089A
:1004A0000F02031C552A071087100C1C08000C10A3
:1004B000C00A851008000C1C72280C10C00B722892
:0A04C0004108C00085018701080013
:084000000100030005000800A7
:02400E00CC33B1
:10420000010078007A007C007E007B0079007F004E
:104210007D007A0078007E007C00FF00FF00FF0038
:104220000000F200F600FA00FE00F200F600FA00CC
:10423000FE00F200F600FA00FE00FF00FF00FF00A3
:10424000010005000500050005000900090009003E
:1042500009000D000D000D000D00FF00FF00FF0024
:10426000FF00FF00FF00FF00FF00FF00FF00FF0056
:10427000FF00FF00FF00FF00FF00FF00FF00FF0046
:10428000FF00FF00FF00FF00FF00FF00FF00FF0036
:10429000FF00FF00FF00FF00FF00FF00FF00FF0026
:1042A000FF00FF00FF00FF00FF00FF00FF00FF0016
:1042B000FF00FF00FF00FF00FF00FF00FF00FF0006
:1042C000FF00FF00FF00FF00FF00FF00FF00FF00F6
:1042D000FF00FF00FF00FF00FF00FF00FF00FF00E6
:1042E000FF00FF00FF00FF00FF00FF00FF00FF00D6
:1042F000FF00FF00FF00FF00FF00FF00FF00DD00E8
:00000001FF
